:020000040000FA
:06000000D6EF03F0120030
:0600080004EF04F01200F9
:060018000CEF04F01200E1
:06002A000100CA070000FE
:08003000800000000200000046
:080038000001776B1E0E716ED2
:100040000401400E096F200E0A6F040E0B6F880E1C
:10005000086F0401200E0E6F040E0F6F400E0C6F20
:100060001200550EA76EAA0EA76EA68212000401FA
:10007000226B010E236F12000001756B41D90AE259
:100080004CD90800F5CF76F0000133D976C0EFFFE8
:10009000752BF4D7F86A1200F00E04012217840EB3
:1000A000A66E0001756B2CD90AE22FD90F0E000144
:1000B00075150F0801E1D5DF0001752BF4D712008B
:1000C000940EA66E0001756B1BD911E27551006E7E
:1000D000016A060ED89000360136E804FBE1026A98
:1000E00001BE0268F7D8BDDF0001752BEDD7F86AB5
:1000F0001200A66A0001756B03D90BE204012251BC
:1001000000017525A96EA680F4D8A8CFEFFF752B46
:10011000F3D712000001756BF3D810E204012251ED
:1001200000017525A96EE5D8EF50A86E040EA66EE5
:1001300098DFA6B2FED70001752BEED71200C40ED1
:10014000A66E0001756BDCD805E2DFD88ADF0001FE
:10015000752BF9D7F86A120097D8060E00017A5D60
:1001600003E36D50020B01E08ED00001770511E131
:1001700004010CBF0DD00401400E096F400E0401B4
:1001800008170401087D880E040108130001776B2D
:100190007AD0040108BF77D00001756B04012051AB
:1001A000320A45E0CD0A34E0F80A2DE0020A26E0E2
:1001B000010A1FE0070A18E0010A11E0030A0AE039
:1001C000070A08E0060A01E04DD051DF0001040EE5
:1001D000756F49D051DF050E0001752744D05CDFF3
:1001E0000001010E756F3FD06BDF0001010E756FCE
:1001F0003AD07FDF050E0001752735D08BDF000177
:10020000010E756F30D09BDF0001010E756F2BD092
:100210006D960001786B796B00017807000E795BB1
:1002200000017851791101E0F7D7FF001CD0030ECF
:100230000401215D09E104012251E8B08C84E8A0A9
:100240008C940001010E756F040E0401215D09E11B
:1002500004012251E8B08C86E8A08C960001010EC2
:10026000756F01D000D00001010E776F000175514C
:100270000AE075C00DF4400E04010C1704010C7D5A
:10028000880E04010C13120000018051811104E159
:10029000200E806F4E0E816F8007000E815B6DA275
:1002A00009D08051811115E18C708C50010B0EE04A
:1002B0008C821200060E00017A5D0BE10001805174
:1002C000811107E18C708C50010B02E08C921200BE
:1002D0008C821200040122510024F36E235101206C
:1002E000F46E24510220F86EF4CFF7FFF3CFF6FF3F
:1002F00012007551EA6A250FE96E040EEA22120017
:10030000040121510001755D1200F3DFEFCF03F00E
:1003100004D803C0F5FF0C00120075C000F0016A9C
:06032000026A6AEF01F021
:0A0326006C5002E0000E01D0010E41
:1003300000090BE0040100513C0BE842E8420D08C3
:1003400002E1AEEF01F0B7EF01F06C5002E0000EF9
:1003500001D0010E040901E019D812000001606B00
:10036000616B666B676B82EC02F039EF02F0020E94
:100370000001605D09E15CD8040100BD02D0C80E37
:1003800001D0880E006F120072EF02F0040E00011F
:100390007A5D09E112C46EFF6E50000802E2050E9C
:1003A00001D0030E7A6F0001600509E10AD804014B
:1003B00004BD02D0C80E01D0880E046F120072EF87
:1003C00002F00001080E665D000E675903E266C088
:1003D00069F002D0080E696F69C005F46951006EBA
:1003E000016A0050665F0150675B180E646F040E6F
:1003F000656F69511CE000017BA307D062C0F6FF66
:1004000063C0F7FF0800F55005D062C0E9FF63C084
:10041000EAFFEF5064C0E9FF65C0EAFFEF6E00013C
:10042000622B000E6323642B65236907E2D7120059
:1004300001C46AF000016A516625666F000E6721EB
:10044000676F180E626F040E636F6A5111E062C02D
:10045000E9FF63C0EAFFEF5064C0E9FF65C0EAFF4F
:10046000EF6E642B000E6523622B63236A07EDD7C2
:1004700012000001615105E13DD8840E006F0401B6
:100480001DD0040110AF1CD0000166510401165D9F
:10049000000167510401175904E216C466F017C43D
:1004A00067F08FDF0001010E606F24D8800E006FAF
:1004B0000401180E066F040E076FC80E046F10D0EB
:1004C0000001020E606F0401056BC80E046F040189
:1004D000080E016F180E026F040E036FC80E006F36
:1004E0006D9812000001606B05D8880E006F040142
:1004F000046B12000401080E016F100E026F040E4F
:04050000036F120073
:0C05040004011051600BE842E842E8429C
:10051000E842E842000901E012001151080A39E0FE
:10052000010A35E00F0A0AE0030A01E012000001A7
:10053000010E616F0001040E7A6F12000001010EBE
:10054000616F0401130507E10001760E626F070E6B
:10055000636F120E13D0020E135D07E10001880EC7
:10056000626F070E636F200E09D0030E135D0AE160
:100570000001A80E626F070E636F040E0001666F24
:10058000676B02D00001616B00017B831200D7EF23
:1005900002F00001010E616F00017C0E626F000E1F
:1005A000636F00017B930001010E666F1200000172
:1005B000010E616F12C47CF00401125104E10001CC
:1005C000050E7A6F12000001060E7A6F1CEF00F024
:1005D000080E6D6E6DBAFED7686A110E696E000165
:1005E000020E7A6F12006850040B06E06950040B8B
:1005F00003E06D92699468946850010B04E06950BF
:10060000010B01E027D86850100B09E06950100B6E
:1006100006E0698468986D82A08A0300A19A6850F8
:10062000200B09E06950200B06E070A003D072ECAB
:1006300002F07090689A030E00017A5D01E209D021
:100640006850080B06E06950080B03E093EC01F0DA
:1006500068961200686A7B0E696E6E6A160E706E7E
:1006600068A602D06896FCD76D9872EC02F0000183
:0A0670007C6B0001030E7A6F12008C
:06067A002A0EF66E000ED0
:10068000F76E000EF86E00010900F550706F09005A
:10069000F550716F03E1706701D03DD00900F5504E
:1006A0006B6F0900F5506C6F0900F5506D6F090014
:1006B0000900F550E96E0900F550EA6E09000900DD
:1006C0000900F5506E6F0900F5506F6F09000900C1
:1006D000F6CF72F0F7CF73F0F8CF74F06BC0F6FF7F
:1006E0006CC0F7FF6DC0F8FF00016E5302E16F535D
:1006F00007E00900F550EE6E6E07F8E26F07F9D7D4
:1007000072C0F6FF73C0F7FF74C0F8FF00017007F6
:08071000000E715BBFD712005F
:08071800C1CF7EF00F0EC112EB
:100720009388A69EFE0EA96EA680A8CF7FF081A812
:1007300008D0FF0E00017F5D04E07EC0C1FF00EF26
:1007400004F0A684FE0EA96EA86A550EA76EAA0E26
:10075000A76EA682A1A8FED7A198F00E8C16F00E67
:100760009516140E6F6EE8EC02F0F3EC02F0ACECB0
:0607700000F0FBD71200AF
:0A0776001201000200000008D80480
:100780000B000000000000010902200001010080B0
:1007900032090400000200000000070501024000C9
:0C07A0000007058102400000040309046A
:0407AC0013EE00F058
:1007B00023EE00F0F86A059C3DEC03F0E4EC03F056
:0807C0008CEC03F0FBD71200E2
:0207C80012001D
:0207CA0000002D
:020000040030CA
:0100000024DB
:010001004EB0
:0100020038C5
:010003001EDE
:010005008179
:010006008178
:0100080000F7
:010009008076
:01000A000FE6
:01000B008074
:01000C000FE4
:01000D0000F2
:00000001FF
